:1000000003C018951895D7C050E0752E852E952EF3
:10001000A52E5CE357BB58BB50E858B951E053BF1D
:1000200050E052BF52E059BF33247724442488243F
:1000300055249924789413C070E084D071E082D064
:1000400021C010E0FF27E3E0E199FECF1EBBE09A5C
:100050005DB350831395E395EF30C1F713C0552777
:10006000FF27EEE0E199FECFEEBBE09A5DB3F50F1E
:10007000EA95EF3FC9F75FE05EBBE09A5DB3F51725
:1000800001F300C079C028F5E72FEF70F0E0707F32
:10009000703171F07032B1F07034E9F0703521F1E7
:1000A0007036F9F1703739F1703831F2703949F240
:1000B000FF27D3E0ED0F2082B22D75D0D4E0ED0FF5
:1000C000B083E0CFFF2753E0E50F708188943AD0EA
:1000D000D9CF272ED7CFE199FECFEEBB2DBAF8941A
:1000E000E29AE19A7894CECFE199FECFEEBBE09A06
:1000F0007DB328D0C7CF5527FF27EEE0E199FECF8B
:10010000EEBBE09A5DB3F50FEA95EF3FC9F7E199D1
:10011000FECFEFE0EEBBFDBBF894E29AE19A789453
:10012000B1CF10E0FF27E3E05081E199FECF1EBB85
:100130005DBBF894E29AE19A78941395E395EF30D9
:1001400099F7D9CF99E0B19BFECFB89810F0C0983D
:10015000B89AC198B99A23D0B99821D0B199F9CF5A
:1001600010F0B89802C0C098B89AB19BFECFB8986A
:10017000771F9A9541F7089599E0B199FECFC198FC
:10018000B99A8894B09B04C00894B099FECF02C07D
:10019000B09BFECFB998771F9A9579F774CF80E41A
:1001A0008A95F1F7089558E0A52FBB1F5795AA959A
:1001B000E1F7B52F08951FB66EE062BF68B36370B4
:1001C0004C7F462B48BB4370C32F3395C327C323B3
:1001D0006C2F672109F044606C2F682109F048609A
:1001E0006C2F692109F040611FBE1895FFFFFFFFCA
:1001F000FFFFFFFFFFFFFFFFFFFFFFFFFFFFFFFF0F
:10020000FFFFFFFFFFFFFFFFFFFFFFFFFFFFFFFFFE
:10021000FFFFFFFFFFFFFFFFFFFFFFFFFFFFFFFFEE
:10022000FFFFFFFFFFFFFFFFFFFFFFFFFFFFFFFFDE
:00000001FF
